
 Start  Stop   Length Name               Class

 00000H 02C91H 02C92H _TEXT              CODE
 02C92H 0338AH 006F9H EX3L_TEXT          CODE
 0338CH 03452H 000C7H OS_CPU_A_TEXT      CODE
 03453H 03538H 000E6H OS_CPU_C_TEXT      CODE
 03539H 0382DH 002F5H PC_TEXT            CODE
 0382EH 04C80H 01453H UCOS_II_TEXT       CODE
 04C90H 05257H 005C8H E87_PROG           CODE
 05260H 05260H 00000H _FARDATA           FAR_DATA
 05260H 05260H 00000H _FARBSS            FAR_BSS
 05260H 05260H 00000H _OVERLAY_          OVRINFO
 05260H 05260H 00000H _1STUB_            STUBSEG
 05260H 05A15H 007B6H _DATA              DATA
 05A16H 05A19H 00004H _CVTSEG            DATA
 05A1AH 05A1FH 00006H _SCNSEG            DATA
 05A20H 05A20H 00000H _CONST             CONST
 05A20H 05A31H 00012H _INIT_             INITDATA
 05A32H 05A32H 00000H _INITEND_          INITDATA
 05A32H 05A37H 00006H _EXIT_             EXITDATA
 05A38H 05A38H 00000H _EXITEND_          EXITDATA
 05A38H 08979H 02F42H _BSS               BSS
 0897AH 0897AH 00000H _BSSEND            BSSEND
 08980H 08A8FH 00110H _STACK             STACK


Detailed map of segments

 0000:0000 0295 C=CODE   S=_TEXT          G=(none)  M=c0.ASM     ACBP=28
 0000:0295 020E C=CODE   S=_TEXT          G=(none)  M=FP87INIT   ACBP=28
 0000:04A3 0000 C=CODE   S=_TEXT          G=(none)  M=E87TRAP    ACBP=28
 0000:04A3 0000 C=CODE   S=_TEXT          G=(none)  M=PROTFLAG   ACBP=28
 0000:04A3 0000 C=CODE   S=_TEXT          G=(none)  M=DEFLT87    ACBP=28
 0000:04A3 01BD C=CODE   S=_TEXT          G=(none)  M=REALCVT    ACBP=28
 0000:0660 020C C=CODE   S=_TEXT          G=(none)  M=XCVT       ACBP=28
 0000:086C 00B1 C=CODE   S=_TEXT          G=(none)  M=FPERR      ACBP=28
 0000:091D 00C9 C=CODE   S=_TEXT          G=(none)  M=_POW10     ACBP=28
 0000:09E6 000B C=CODE   S=_TEXT          G=(none)  M=POW10D     ACBP=28
 0000:09F1 002D C=CODE   S=_TEXT          G=(none)  M=ATEXIT     ACBP=28
 0000:0A1E 0093 C=CODE   S=_TEXT          G=(none)  M=EXIT       ACBP=28
 0000:0AB1 0000 C=CODE   S=_TEXT          G=(none)  M=FILES      ACBP=28
 0000:0AB1 0000 C=CODE   S=_TEXT          G=(none)  M=FILES2     ACBP=28
 0000:0AB1 0000 C=CODE   S=_TEXT          G=(none)  M=FPSTKLEN   ACBP=28
 0000:0AB1 0017 C=CODE   S=_TEXT          G=(none)  M=F_LXMUL    ACBP=28
 0000:0AC8 001C C=CODE   S=_TEXT          G=(none)  M=F_SCOPY    ACBP=28
 0000:0AE4 0026 C=CODE   S=_TEXT          G=(none)  M=GETDATE    ACBP=28
 0000:0B0A 0020 C=CODE   S=_TEXT          G=(none)  M=GETVECT    ACBP=28
 0000:0B2A 00AE C=CODE   S=_TEXT          G=(none)  M=H_LDIV     ACBP=28
 0000:0BD8 0021 C=CODE   S=_TEXT          G=(none)  M=H_LLSH     ACBP=28
 0000:0BF9 0060 C=CODE   S=_TEXT          G=(none)  M=H_PADD     ACBP=28
 0000:0C59 004B C=CODE   S=_TEXT          G=(none)  M=IOERROR    ACBP=28
 0000:0CA4 0011 C=CODE   S=_TEXT          G=(none)  M=ISATTY     ACBP=28
 0000:0CB5 00A2 C=CODE   S=_TEXT          G=(none)  M=LONGTOA    ACBP=28
 0000:0D57 0029 C=CODE   S=_TEXT          G=(none)  M=LSEEK      ACBP=28
 0000:0D80 0021 C=CODE   S=_TEXT          G=(none)  M=N_PCMP     ACBP=28
 0000:0DA1 00BA C=CODE   S=_TEXT          G=(none)  M=SETUPIO    ACBP=28
 0000:0E5B 0000 C=CODE   S=_TEXT          G=(none)  M=SIGDATA    ACBP=28
 0000:0E5B 0000 C=CODE   S=_TEXT          G=(none)  M=STKLEN     ACBP=28
 0000:0E5B 04DB C=CODE   S=_TEXT          G=(none)  M=VPRINTER   ACBP=28
 0000:1336 009F C=CODE   S=_TEXT          G=(none)  M=VRAM       ACBP=28
 0000:13D5 0000 C=CODE   S=_TEXT          G=(none)  M=WSCROLL    ACBP=28
 0000:13D5 014E C=CODE   S=_TEXT          G=(none)  M=CPRINTF    ACBP=28
 0000:1523 01A5 C=CODE   S=_TEXT          G=(none)  M=CRTINIT    ACBP=28
 0000:16C8 001F C=CODE   S=_TEXT          G=(none)  M=CVTFAK     ACBP=28
 0000:16E7 0432 C=CODE   S=_TEXT          G=(none)  M=FARHEAP    ACBP=28
 0000:1B19 0140 C=CODE   S=_TEXT          G=(none)  M=FBRK       ACBP=28
 0000:1C59 005E C=CODE   S=_TEXT          G=(none)  M=GETCH      ACBP=28
 0000:1CB7 00AC C=CODE   S=_TEXT          G=(none)  M=GPTEXT     ACBP=28
 0000:1D63 0012 C=CODE   S=_TEXT          G=(none)  M=KBHIT      ACBP=28
 0000:1D75 009D C=CODE   S=_TEXT          G=(none)  M=MOVETEXT   ACBP=28
 0000:1E12 0017 C=CODE   S=_TEXT          G=(none)  M=PUTCH      ACBP=28
 0000:1E29 0004 C=CODE   S=_TEXT          G=(none)  M=REALCVT    ACBP=28
 0000:1E2D 01C7 C=CODE   S=_TEXT          G=(none)  M=SCREEN     ACBP=28
 0000:1FF4 018E C=CODE   S=_TEXT          G=(none)  M=SCROLL     ACBP=28
 0000:2182 001C C=CODE   S=_TEXT          G=(none)  M=SETBLOCK   ACBP=28
 0000:219E 006A C=CODE   S=_TEXT          G=(none)  M=SETJMP     ACBP=28
 0000:2208 002C C=CODE   S=_TEXT          G=(none)  M=WHEREXY    ACBP=28
 0000:2234 00CD C=CODE   S=_TEXT          G=(none)  M=FFLUSH     ACBP=28
 0000:2301 0042 C=CODE   S=_TEXT          G=(none)  M=FLUSHALL   ACBP=28
 0000:2343 001C C=CODE   S=_TEXT          G=(none)  M=FPRINTF    ACBP=28
 0000:235F 01E2 C=CODE   S=_TEXT          G=(none)  M=FSEEK      ACBP=28
 0000:2541 0024 C=CODE   S=_TEXT          G=(none)  M=MEMCPY     ACBP=28
 0000:2565 03C8 C=CODE   S=_TEXT          G=(none)  M=PUTC       ACBP=28
 0000:292D 011D C=CODE   S=_TEXT          G=(none)  M=SETVBUF    ACBP=28
 0000:2A4A 0083 C=CODE   S=_TEXT          G=(none)  M=SPRINTF    ACBP=28
 0000:2ACD 0151 C=CODE   S=_TEXT          G=(none)  M=WRITE      ACBP=28
 0000:2C1E 003C C=CODE   S=_TEXT          G=(none)  M=WRITEA     ACBP=28
 0000:2C5A 0038 C=CODE   S=_TEXT          G=(none)  M=XFFLUSH    ACBP=28
 02C9:0002 06F9 C=CODE   S=EX3L_TEXT      G=(none)  M=EX3L.C     ACBP=28
 0338:000C 00C7 C=CODE   S=OS_CPU_A_TEXT  G=(none)  M=..\IX86L\OS_CPU_A.ASM ACBP=48
 0345:0003 00E6 C=CODE   S=OS_CPU_C_TEXT  G=(none)  M=..\IX86L\OS_CPU_C.C ACBP=28
 0353:0009 02F5 C=CODE   S=PC_TEXT        G=(none)  M=..\..\BLOCKS\PC\SOURCE\PC.C ACBP=28
 0382:000E 1453 C=CODE   S=UCOS_II_TEXT   G=(none)  M=..\SOURCE\UCOS_II.C ACBP=28
 04C9:0000 0000 C=CODE   S=E87_PROG       G=(none)  M=FP87INIT   ACBP=68
 04C9:0000 03E3 C=CODE   S=E87_PROG       G=(none)  M=EMU087     ACBP=68
 04C9:03F0 01D8 C=CODE   S=E87_PROG       G=(none)  M=E87TRAP    ACBP=68
 0526:0000 0000 C=FAR_DATA S=_FARDATA       G=(none)  M=c0.ASM     ACBP=68
 0526:0000 0000 C=FAR_BSS S=_FARBSS        G=(none)  M=c0.ASM     ACBP=68
 0526:0000 0000 C=OVRINFO S=_OVERLAY_      G=(none)  M=c0.ASM     ACBP=68
 0526:0000 0000 C=STUBSEG S=_1STUB_        G=(none)  M=c0.ASM     ACBP=68
 0526:0000 0093 C=DATA   S=_DATA          G=DGROUP  M=c0.ASM     ACBP=68
 0526:0094 01E1 C=DATA   S=_DATA          G=DGROUP  M=EX3L.C     ACBP=48
 0526:0276 0000 C=DATA   S=_DATA          G=DGROUP  M=..\IX86L\OS_CPU_A.ASM ACBP=48
 0526:0276 0000 C=DATA   S=_DATA          G=DGROUP  M=..\IX86L\OS_CPU_C.C ACBP=48
 0526:0276 001F C=DATA   S=_DATA          G=DGROUP  M=..\..\BLOCKS\PC\SOURCE\PC.C ACBP=48
 0526:0296 0108 C=DATA   S=_DATA          G=DGROUP  M=..\SOURCE\UCOS_II.C ACBP=48
 0526:03A0 0002 C=DATA   S=_DATA          G=DGROUP  M=FP87INIT   ACBP=68
 0526:03B0 0000 C=DATA   S=_DATA          G=DGROUP  M=E87TRAP    ACBP=68
 0526:03B0 0003 C=DATA   S=_DATA          G=DGROUP  M=PROTFLAG   ACBP=48
 0526:03B4 0002 C=DATA   S=_DATA          G=DGROUP  M=DEFLT87    ACBP=48
 0526:03B6 0000 C=DATA   S=_DATA          G=DGROUP  M=REALCVT    ACBP=48
 0526:03B6 0000 C=DATA   S=_DATA          G=DGROUP  M=XCVT       ACBP=48
 0526:03B6 009A C=DATA   S=_DATA          G=DGROUP  M=FPERR      ACBP=48
 0526:0450 0080 C=DATA   S=_DATA          G=DGROUP  M=_POW10     ACBP=48
 0526:04D0 0000 C=DATA   S=_DATA          G=DGROUP  M=POW10D     ACBP=48
 0526:04D0 0002 C=DATA   S=_DATA          G=DGROUP  M=ATEXIT     ACBP=48
 0526:04D2 000C C=DATA   S=_DATA          G=DGROUP  M=EXIT       ACBP=48
 0526:04DE 0190 C=DATA   S=_DATA          G=DGROUP  M=FILES      ACBP=48
 0526:066E 002A C=DATA   S=_DATA          G=DGROUP  M=FILES2     ACBP=48
 0526:0698 0002 C=DATA   S=_DATA          G=DGROUP  M=FPSTKLEN   ACBP=48
 0526:069A 0000 C=DATA   S=_DATA          G=DGROUP  M=F_LXMUL    ACBP=48
 0526:069A 0000 C=DATA   S=_DATA          G=DGROUP  M=F_SCOPY    ACBP=48
 0526:069A 0000 C=DATA   S=_DATA          G=DGROUP  M=GETDATE    ACBP=48
 0526:069A 0000 C=DATA   S=_DATA          G=DGROUP  M=GETVECT    ACBP=48
 0526:069A 0000 C=DATA   S=_DATA          G=DGROUP  M=H_LDIV     ACBP=48
 0526:069A 0000 C=DATA   S=_DATA          G=DGROUP  M=H_LLSH     ACBP=48
 0526:069A 0000 C=DATA   S=_DATA          G=DGROUP  M=H_PADD     ACBP=48
 0526:069A 005B C=DATA   S=_DATA          G=DGROUP  M=IOERROR    ACBP=48
 0526:06F6 0000 C=DATA   S=_DATA          G=DGROUP  M=ISATTY     ACBP=48
 0526:06F6 0000 C=DATA   S=_DATA          G=DGROUP  M=LONGTOA    ACBP=48
 0526:06F6 0000 C=DATA   S=_DATA          G=DGROUP  M=LSEEK      ACBP=48
 0526:06F6 0000 C=DATA   S=_DATA          G=DGROUP  M=N_PCMP     ACBP=48
 0526:06F6 0000 C=DATA   S=_DATA          G=DGROUP  M=SETUPIO    ACBP=48
 0526:06F6 0000 C=DATA   S=_DATA          G=DGROUP  M=SIGDATA    ACBP=48
 0526:06F6 0002 C=DATA   S=_DATA          G=DGROUP  M=STKLEN     ACBP=48
 0526:06F8 0067 C=DATA   S=_DATA          G=DGROUP  M=VPRINTER   ACBP=48
 0526:0760 0000 C=DATA   S=_DATA          G=DGROUP  M=VRAM       ACBP=48
 0526:0760 0002 C=DATA   S=_DATA          G=DGROUP  M=WSCROLL    ACBP=48
 0526:0762 0000 C=DATA   S=_DATA          G=DGROUP  M=CPRINTF    ACBP=48
 0526:0762 0018 C=DATA   S=_DATA          G=DGROUP  M=CRTINIT    ACBP=48
 0526:077A 0031 C=DATA   S=_DATA          G=DGROUP  M=CVTFAK     ACBP=48
 0526:07AC 0000 C=DATA   S=_DATA          G=DGROUP  M=FARHEAP    ACBP=48
 0526:07AC 0002 C=DATA   S=_DATA          G=DGROUP  M=FBRK       ACBP=48
 0526:07AE 0000 C=DATA   S=_DATA          G=DGROUP  M=GETCH      ACBP=48
 0526:07AE 0000 C=DATA   S=_DATA          G=DGROUP  M=GPTEXT     ACBP=48
 0526:07AE 0002 C=DATA   S=_DATA          G=DGROUP  M=KBHIT      ACBP=48
 0526:07B0 0000 C=DATA   S=_DATA          G=DGROUP  M=MOVETEXT   ACBP=48
 0526:07B0 0000 C=DATA   S=_DATA          G=DGROUP  M=PUTCH      ACBP=48
 0526:07B0 0000 C=DATA   S=_DATA          G=DGROUP  M=REALCVT    ACBP=48
 0526:07B0 0000 C=DATA   S=_DATA          G=DGROUP  M=SCREEN     ACBP=48
 0526:07B0 0000 C=DATA   S=_DATA          G=DGROUP  M=SCROLL     ACBP=48
 0526:07B0 0000 C=DATA   S=_DATA          G=DGROUP  M=SETBLOCK   ACBP=48
 0526:07B0 0000 C=DATA   S=_DATA          G=DGROUP  M=SETJMP     ACBP=48
 0526:07B0 0000 C=DATA   S=_DATA          G=DGROUP  M=WHEREXY    ACBP=48
 0526:07B0 0000 C=DATA   S=_DATA          G=DGROUP  M=FFLUSH     ACBP=48
 0526:07B0 0000 C=DATA   S=_DATA          G=DGROUP  M=FLUSHALL   ACBP=48
 0526:07B0 0000 C=DATA   S=_DATA          G=DGROUP  M=FPRINTF    ACBP=48
 0526:07B0 0000 C=DATA   S=_DATA          G=DGROUP  M=FSEEK      ACBP=48
 0526:07B0 0000 C=DATA   S=_DATA          G=DGROUP  M=MEMCPY     ACBP=48
 0526:07B0 0001 C=DATA   S=_DATA          G=DGROUP  M=PUTC       ACBP=48
 0526:07B2 0004 C=DATA   S=_DATA          G=DGROUP  M=SETVBUF    ACBP=48
 0526:07B6 0000 C=DATA   S=_DATA          G=DGROUP  M=SPRINTF    ACBP=48
 0526:07B6 0000 C=DATA   S=_DATA          G=DGROUP  M=WRITE      ACBP=48
 0526:07B6 0000 C=DATA   S=_DATA          G=DGROUP  M=WRITEA     ACBP=48
 0526:07B6 0000 C=DATA   S=_DATA          G=DGROUP  M=XFFLUSH    ACBP=48
 0526:07B6 0000 C=DATA   S=_CVTSEG        G=DGROUP  M=c0.ASM     ACBP=48
 0526:07B6 0002 C=DATA   S=_CVTSEG        G=DGROUP  M=REALCVT    ACBP=48
 0526:07B8 0002 C=DATA   S=_CVTSEG        G=DGROUP  M=CVTFAK     ACBP=48
 0526:07BA 0000 C=DATA   S=_CVTSEG        G=DGROUP  M=REALCVT    ACBP=48
 0526:07BA 0000 C=DATA   S=_SCNSEG        G=DGROUP  M=c0.ASM     ACBP=48
 0526:07BA 0006 C=DATA   S=_SCNSEG        G=DGROUP  M=CVTFAK     ACBP=48
 0526:07C0 0000 C=CONST  S=_CONST         G=DGROUP  M=c0.ASM     ACBP=48
 0526:07C0 0000 C=INITDATA S=_INIT_         G=DGROUP  M=c0.ASM     ACBP=48
 0526:07C0 0006 C=INITDATA S=_INIT_         G=DGROUP  M=FP87INIT   ACBP=48
 0526:07C6 0006 C=INITDATA S=_INIT_         G=DGROUP  M=SETUPIO    ACBP=48
 0526:07CC 0006 C=INITDATA S=_INIT_         G=DGROUP  M=CRTINIT    ACBP=48
 0526:07D2 0000 C=INITDATA S=_INITEND_      G=DGROUP  M=c0.ASM     ACBP=28
 0526:07D2 0000 C=EXITDATA S=_EXIT_         G=DGROUP  M=c0.ASM     ACBP=48
 0526:07D2 0006 C=EXITDATA S=_EXIT_         G=DGROUP  M=FP87INIT   ACBP=48
 0526:07D8 0000 C=EXITDATA S=_EXITEND_      G=DGROUP  M=c0.ASM     ACBP=28
 0526:07D8 0000 C=BSS    S=_BSS           G=DGROUP  M=c0.ASM     ACBP=48
 0526:07D8 1DD0 C=BSS    S=_BSS           G=DGROUP  M=EX3L.C     ACBP=48
 0526:25A8 0001 C=BSS    S=_BSS           G=DGROUP  M=..\IX86L\OS_CPU_C.C ACBP=48
 0526:25AA 001B C=BSS    S=_BSS           G=DGROUP  M=..\..\BLOCKS\PC\SOURCE\PC.C ACBP=48
 0526:25C6 10CE C=BSS    S=_BSS           G=DGROUP  M=..\SOURCE\UCOS_II.C ACBP=48
 0526:3694 0000 C=BSS    S=_BSS           G=DGROUP  M=REALCVT    ACBP=48
 0526:3694 0000 C=BSS    S=_BSS           G=DGROUP  M=XCVT       ACBP=48
 0526:3694 0000 C=BSS    S=_BSS           G=DGROUP  M=_POW10     ACBP=48
 0526:3694 0080 C=BSS    S=_BSS           G=DGROUP  M=ATEXIT     ACBP=48
 0526:3714 0000 C=BSS    S=_BSS           G=DGROUP  M=GETVECT    ACBP=48
 0526:3714 0000 C=BSS    S=_BSS           G=DGROUP  M=IOERROR    ACBP=48
 0526:3714 0000 C=BSS    S=_BSS           G=DGROUP  M=ISATTY     ACBP=48
 0526:3714 0000 C=BSS    S=_BSS           G=DGROUP  M=LONGTOA    ACBP=48
 0526:3714 0000 C=BSS    S=_BSS           G=DGROUP  M=LSEEK      ACBP=48
 0526:3714 0000 C=BSS    S=_BSS           G=DGROUP  M=SETUPIO    ACBP=48
 0526:3714 0004 C=BSS    S=_BSS           G=DGROUP  M=SIGDATA    ACBP=48
 0526:3718 0000 C=BSS    S=_BSS           G=DGROUP  M=VPRINTER   ACBP=48
 0526:3718 0000 C=BSS    S=_BSS           G=DGROUP  M=VRAM       ACBP=48
 0526:3718 0000 C=BSS    S=_BSS           G=DGROUP  M=CRTINIT    ACBP=48
 0526:3718 0000 C=BSS    S=_BSS           G=DGROUP  M=GETCH      ACBP=48
 0526:3718 0000 C=BSS    S=_BSS           G=DGROUP  M=KBHIT      ACBP=48
 0526:3718 0000 C=BSS    S=_BSS           G=DGROUP  M=SETBLOCK   ACBP=48
 0526:3718 0000 C=BSS    S=_BSS           G=DGROUP  M=SETJMP     ACBP=48
 0526:3718 0000 C=BSS    S=_BSS           G=DGROUP  M=MEMCPY     ACBP=48
 0526:3718 0001 C=BSS    S=_BSS           G=DGROUP  M=PUTC       ACBP=48
 0526:371A 0000 C=BSS    S=_BSS           G=DGROUP  M=WRITEA     ACBP=48
 0526:371A 0000 C=BSSEND S=_BSSEND        G=DGROUP  M=c0.ASM     ACBP=28
 0898:0000 0110 C=STACK  S=_STACK         G=(none)  M=c0.ASM     ACBP=74
 0898:0000 0080 C=STACK  S=_STACK         G=(none)  M=EMUVARS    ACBP=78

  Address         Publics by Name

 0526:0000 idle  DATASEG@
 0000:0291 idle  DGROUP@
 04C9:0306       e087_Entry
 04C9:03C6       e087_Shortcut
 04C9:0430       e087_Trap
 0000:0000 idle  FIARQQ
 0000:0000 idle  FICRQQ
 0000:0000  Abs  FIDRQQ
 0000:0000  Abs  FIERQQ
 0000:0000 idle  FISRQQ
 0000:0000  Abs  FIWRQQ
 0000:0000 idle  FJARQQ
 0000:0000 idle  FJCRQQ
 0000:0000 idle  FJSRQQ
 0000:0B2D idle  F_LDIV@
 0000:0B3C idle  F_LMOD@
 0000:0B34       F_LUDIV@
 0000:0B44 idle  F_LUMOD@
 0000:0BDB idle  F_LXLSH@
 0000:0AB1       F_LXMUL@
 0000:0BFC idle  F_PADD@
 0000:0C2B idle  F_PSUB@
 0000:0AC8       F_SCOPY@
 0000:0B2D idle  LDIV@
 0000:0B3C idle  LMOD@
 0000:0B34 idle  LUDIV@
 0000:0B44 idle  LUMOD@
 0000:0BDB idle  LXLSH@
 0000:0AB1 idle  LXMUL@
 0000:0B2A idle  N_LDIV@
 0000:0B39 idle  N_LMOD@
 0000:0B31 idle  N_LUDIV@
 0000:0B41 idle  N_LUMOD@
 0000:0BD8       N_LXLSH@
 0000:0BF9       N_PADD@
 0000:0D80       N_PCMP@
 0000:0C28 idle  N_PSUB@
 0000:0BFC idle  PADD@
 0000:0C2B idle  PSUB@
 0000:0AC8 idle  SCOPY@
 0000:027A       _abort
 0000:09F1 idle  _atexit
 0000:1507 idle  _cprintf
 0526:0771       _directvideo
 02C9:052A idle  _DispTaskStat
 0526:007F       _errno
 0000:0A76       _exit
 0000:1827 idle  _farfree
 0000:193B idle  _farmalloc
 0000:1A9F idle  _farrealloc
 0000:2234       _fflush
 0000:2301       _flushall
 0000:2343       _fprintf
 0000:2581 idle  _fputc
 0000:2716 idle  _fputchar
 0000:1827       _free
 0000:23E1       _fseek
 0000:2461 idle  _ftell
 0000:1C59       _getch
 0000:1C75 idle  _getche
 0000:0AE4       _getdate
 0000:1CB7       _gettext
 0000:0AF7       _gettime
 0000:0B0A       _getvect
 0000:0CA4       _isatty
 0000:1D63       _kbhit
 0000:21D4       _longjmp
 0000:0D57       _lseek
 02C9:0002       _main
 0000:1931       _malloc
 0000:2541       _memcpy
 0000:1D75       _movetext
 0526:0828 idle  _MsgQueue
 0526:07D8 idle  _MsgQueueTbl
 0526:3547       _OSCPUUsage
 0338:0029       _OSCtxSw
 0526:3690       _OSCtxSwCtr
 0526:368C idle  _OSEventFreeList
 0382:000E idle  _OSEventTaskRdy
 0382:00D8 idle  _OSEventTaskWait
 0526:354C idle  _OSEventTbl
 0382:0145 idle  _OSEventTO
 0382:0199 idle  _OSEventWaitListInit
 0526:3548 idle  _OSIdleCtr
 0526:3543 idle  _OSIdleCtrMax
 0526:353F idle  _OSIdleCtrRun
 0382:01BD       _OSInit
 0338:0064       _OSIntCtxSw
 0382:032A idle  _OSIntEnter
 0382:0332       _OSIntExit
 0526:353D       _OSIntNesting
 0526:353C idle  _OSLockNesting
 0526:0296 idle  _OSMapTbl
 0382:079D idle  _OSMboxAccept
 0382:07E2       _OSMboxCreate
 0382:0843       _OSMboxPend
 0382:096B       _OSMboxPost
 0382:09CB idle  _OSMboxQuery
 0526:353B       _OSPrioCur
 0526:353A       _OSPrioHighRdy
 0382:0A42 idle  _OSQAccept
 0382:0AD4       _OSQCreate
 0382:0BE9 idle  _OSQFlush
 0382:0C36 idle  _OSQInit
 0382:0C6B       _OSQPend
 0382:0E04       _OSQPost
 0382:0EB3 idle  _OSQPostFront
 0382:0F5E idle  _OSQQuery
 0526:3539 idle  _OSRdyGrp
 0526:3531 idle  _OSRdyTbl
 0526:3530       _OSRunning
 0382:039D idle  _OSSched
 0382:03FD idle  _OSSchedLock
 0382:040C idle  _OSSchedUnlock
 0382:0435       _OSStart
 0338:000C       _OSStartHighRdy
 0382:0494       _OSStatInit
 0526:353E idle  _OSStatRdy
 0382:101A       _OSTaskCreateExt
 02C9:05B9       _OSTaskCreateHook
 0526:352F       _OSTaskCtr
 02C9:05BE idle  _OSTaskDelHook
 0382:04CF idle  _OSTaskIdle
 0382:1218 idle  _OSTaskQuery
 0382:04EF idle  _OSTaskStat
 02C9:0607       _OSTaskStatHook
 0382:1133 idle  _OSTaskStkChk
 0345:0003       _OSTaskStkInit
 02C9:05C3       _OSTaskSwHook
 0526:352B       _OSTCBCur
 0526:3527 idle  _OSTCBFreeList
 0526:3523       _OSTCBHighRdy
 0382:05AA idle  _OSTCBInit
 0526:351F idle  _OSTCBList
 0526:341F idle  _OSTCBPrioTbl
 0526:25A8       _OSTickDOSCtr
 0338:009F       _OSTickISR
 0526:341B idle  _OSTime
 0382:127B       _OSTimeDly
 0382:12C2       _OSTimeDlyHMSM
 0382:13B1 idle  _OSTimeDlyResume
 0382:142D idle  _OSTimeGet
 0382:144C idle  _OSTimeSet
 0382:070E       _OSTimeTick
 02C9:06FA       _OSTimeTickHook
 0526:029E idle  _OSUnMapTbl
 0382:0799       _OSVersion
 0353:0073       _PC_DispChar
 0353:003A idle  _PC_DispClrLine
 0353:0009       _PC_DispClrScr
 0353:00B1       _PC_DispStr
 0353:0100       _PC_DOSReturn
 0353:0114       _PC_DOSSaveReturn
 0353:018B       _PC_ElapsedInit
 0353:019F       _PC_ElapsedStart
 0353:01C2       _PC_ElapsedStop
 0353:0210       _PC_GetDateTime
 0353:0263       _PC_GetKey
 0353:028A       _PC_SetTickRate
 0526:25AA idle  _PC_TickISR
 0353:02D2 idle  _PC_VectGet
 0353:02E5       _PC_VectSet
 0000:09E6       _pow10
 0000:1E12       _putch
 0000:1D0D       _puttext
 0000:1A98 idle  _realloc
 0000:2182       _setblock
 0000:219E       _setjmp
 0000:292D       _setvbuf
 0000:0B19       _setvect
 0000:2A8A       _sprintf
 02C9:039F idle  _Task1
 0526:182C idle  _Task1Stk
 02C9:0425 idle  _Task2
 0526:142C idle  _Task2Stk
 02C9:0472 idle  _Task3
 0526:102C idle  _Task3Stk
 02C9:04C6 idle  _Task4
 0526:0C2C idle  _Task4Stk
 02C9:0519 idle  _Task5
 0526:082C idle  _Task5Stk
 02C9:057F idle  _TaskClk
 0526:1C2C idle  _TaskClkStk
 02C9:006C idle  _TaskStart
 0526:202C idle  _TaskStartStk
 0526:242C idle  _TaskUserData
 0000:1C99 idle  _ungetch
 0000:2AAC idle  _vsprintf
 0000:2212 idle  _wherex
 0000:2221 idle  _wherey
 0526:03A0 idle  __8087
 0000:1000 idle  __AHINCR
 0000:000C idle  __AHSHIFT
 0526:04D0       __atexitcnt
 0526:3694       __atexittbl
 0000:1B8F       __brk
 0526:008B       __brklvl
 0526:006B idle  __C0argc
 0526:006D idle  __C0argv
 0000:15E9 idle  __c0crtinit
 0526:0071 idle  __C0environ
 0526:07AF       __cChar
 0000:0A97 idle  __cexit
 0526:07AE       __cFlag
 0000:016A       __checknull
 0000:0157       __cleanup
 0000:13D5       __CPUTN
 0000:1606 idle  __crtinit
 0000:0000  Abs  __cvtfak
 0000:0AA5 idle  __c_exit
 0526:03B4       __default87
 0526:069A idle  __doserrno
 0000:0C92 idle  __DOSERROR
 0526:069C idle  __dosErrorToSV
 0898:0000       __emu
 0526:0075 idle  __envLng
 0526:0077 idle  __envseg
 0526:0079 idle  __envSize
 0000:0A85       __exit
 0526:04D2       __exitbuf
 0526:04D6 idle  __exitfopen
 0526:04DA idle  __exitopen
 0000:086C       __fperror
 0526:0698       __fpstklen
 0000:049F idle  __fpuint
 0000:2565 idle  __fputc
 0000:272A       __FPUTN
 0526:0087       __heapbase
 0526:008F       __heaptop
 0526:005B idle  __Int0Vector
 0526:005F idle  __Int4Vector
 0526:0063 idle  __Int5Vector
 0526:0067 idle  __Int6Vector
 0000:0C59       __IOERROR
 0526:03B1       __LDT
 0000:0CB5       __LONGTOA
 0000:0293 idle  __MMODEL
 0526:066E       __nfile
 0000:1C72 idle  __Ngetche
 0000:1C96 idle  __Nungetch
 0526:0670       __openfd
 0526:007D idle  __osmajor
 0526:007E idle  __osminor
 0526:007D idle  __osversion
 0000:091D       __POW10
 0526:03B0       __protected
 0526:007B       __psp
 0000:1E29       __REALCVT
 0526:07B6       __RealCvtVector
 0000:01C0       __restorezero
 0000:1BCE       __sbrk
 0526:07BA idle  __ScanTodVector
 0000:1F63       __SCREENIO
 0000:2016       __SCROLL
 0000:0DA1       __setupio
 0526:0081 idle  __StartTime
 0526:06F6       __stklen
 0526:04DE       __streams
 0000:016B       __terminate
 0000:0000 idle  __turboCrt
 0000:0000  Abs  __turboCvt
 0000:0D37 idle  __UTOA
 0000:1F9F       __VALIDATEXY
 0526:007D       __version
 0526:0762       __video
 0000:155E       __VideoInt
 0000:0E73       __VPRINTER
 0000:1336       __VPTR
 0000:135B       __VRAM
 0000:2208       __wherexy
 0000:2C1E       __write
 0526:0760       __wscroll
 0000:0660       __XCVT
 0000:2C5A       __xfflush
 0526:0085 idle  ___brklvl
 0000:16E7 idle  ___first
 0000:03CE idle  ___fpreset
 0000:16E9 idle  ___last
 0000:16EB idle  ___rover
 0526:3714       ___SignalPtr
 0000:2ACD       ___write

  Address         Publics by Value

 0000:0000  Abs  FIWRQQ
 0000:0000  Abs  FIDRQQ
 0000:0000  Abs  __turboCvt
 0000:0000 idle  FIARQQ
 0000:0000 idle  FICRQQ
 0000:0000 idle  FISRQQ
 0000:0000  Abs  FIERQQ
 0000:0000 idle  FJARQQ
 0000:0000 idle  FJCRQQ
 0000:0000 idle  FJSRQQ
 0000:0000 idle  __turboCrt
 0000:0000  Abs  __cvtfak
 0000:000C idle  __AHSHIFT
 0000:0157       __cleanup
 0000:016A       __checknull
 0000:016B       __terminate
 0000:01C0       __restorezero
 0000:027A       _abort
 0000:0291 idle  DGROUP@
 0000:0293 idle  __MMODEL
 0000:03CE idle  ___fpreset
 0000:049F idle  __fpuint
 0000:0660       __XCVT
 0000:086C       __fperror
 0000:091D       __POW10
 0000:09E6       _pow10
 0000:09F1 idle  _atexit
 0000:0A76       _exit
 0000:0A85       __exit
 0000:0A97 idle  __cexit
 0000:0AA5 idle  __c_exit
 0000:0AB1       F_LXMUL@
 0000:0AB1 idle  LXMUL@
 0000:0AC8       F_SCOPY@
 0000:0AC8 idle  SCOPY@
 0000:0AE4       _getdate
 0000:0AF7       _gettime
 0000:0B0A       _getvect
 0000:0B19       _setvect
 0000:0B2A idle  N_LDIV@
 0000:0B2D idle  LDIV@
 0000:0B2D idle  F_LDIV@
 0000:0B31 idle  N_LUDIV@
 0000:0B34       F_LUDIV@
 0000:0B34 idle  LUDIV@
 0000:0B39 idle  N_LMOD@
 0000:0B3C idle  F_LMOD@
 0000:0B3C idle  LMOD@
 0000:0B41 idle  N_LUMOD@
 0000:0B44 idle  LUMOD@
 0000:0B44 idle  F_LUMOD@
 0000:0BD8       N_LXLSH@
 0000:0BDB idle  LXLSH@
 0000:0BDB idle  F_LXLSH@
 0000:0BF9       N_PADD@
 0000:0BFC idle  F_PADD@
 0000:0BFC idle  PADD@
 0000:0C28 idle  N_PSUB@
 0000:0C2B idle  F_PSUB@
 0000:0C2B idle  PSUB@
 0000:0C59       __IOERROR
 0000:0C92 idle  __DOSERROR
 0000:0CA4       _isatty
 0000:0CB5       __LONGTOA
 0000:0D37 idle  __UTOA
 0000:0D57       _lseek
 0000:0D80       N_PCMP@
 0000:0DA1       __setupio
 0000:0E73       __VPRINTER
 0000:1000 idle  __AHINCR
 0000:1336       __VPTR
 0000:135B       __VRAM
 0000:13D5       __CPUTN
 0000:1507 idle  _cprintf
 0000:155E       __VideoInt
 0000:15E9 idle  __c0crtinit
 0000:1606 idle  __crtinit
 0000:16E7 idle  ___first
 0000:16E9 idle  ___last
 0000:16EB idle  ___rover
 0000:1827       _free
 0000:1827 idle  _farfree
 0000:1931       _malloc
 0000:193B idle  _farmalloc
 0000:1A98 idle  _realloc
 0000:1A9F idle  _farrealloc
 0000:1B8F       __brk
 0000:1BCE       __sbrk
 0000:1C59       _getch
 0000:1C72 idle  __Ngetche
 0000:1C75 idle  _getche
 0000:1C96 idle  __Nungetch
 0000:1C99 idle  _ungetch
 0000:1CB7       _gettext
 0000:1D0D       _puttext
 0000:1D63       _kbhit
 0000:1D75       _movetext
 0000:1E12       _putch
 0000:1E29       __REALCVT
 0000:1F63       __SCREENIO
 0000:1F9F       __VALIDATEXY
 0000:2016       __SCROLL
 0000:2182       _setblock
 0000:219E       _setjmp
 0000:21D4       _longjmp
 0000:2208       __wherexy
 0000:2212 idle  _wherex
 0000:2221 idle  _wherey
 0000:2234       _fflush
 0000:2301       _flushall
 0000:2343       _fprintf
 0000:23E1       _fseek
 0000:2461 idle  _ftell
 0000:2541       _memcpy
 0000:2565 idle  __fputc
 0000:2581 idle  _fputc
 0000:2716 idle  _fputchar
 0000:272A       __FPUTN
 0000:292D       _setvbuf
 0000:2A8A       _sprintf
 0000:2AAC idle  _vsprintf
 0000:2ACD       ___write
 0000:2C1E       __write
 0000:2C5A       __xfflush
 02C9:0002       _main
 02C9:006C idle  _TaskStart
 02C9:039F idle  _Task1
 02C9:0425 idle  _Task2
 02C9:0472 idle  _Task3
 02C9:04C6 idle  _Task4
 02C9:0519 idle  _Task5
 02C9:052A idle  _DispTaskStat
 02C9:057F idle  _TaskClk
 02C9:05B9       _OSTaskCreateHook
 02C9:05BE idle  _OSTaskDelHook
 02C9:05C3       _OSTaskSwHook
 02C9:0607       _OSTaskStatHook
 02C9:06FA       _OSTimeTickHook
 0338:000C       _OSStartHighRdy
 0338:0029       _OSCtxSw
 0338:0064       _OSIntCtxSw
 0338:009F       _OSTickISR
 0345:0003       _OSTaskStkInit
 0353:0009       _PC_DispClrScr
 0353:003A idle  _PC_DispClrLine
 0353:0073       _PC_DispChar
 0353:00B1       _PC_DispStr
 0353:0100       _PC_DOSReturn
 0353:0114       _PC_DOSSaveReturn
 0353:018B       _PC_ElapsedInit
 0353:019F       _PC_ElapsedStart
 0353:01C2       _PC_ElapsedStop
 0353:0210       _PC_GetDateTime
 0353:0263       _PC_GetKey
 0353:028A       _PC_SetTickRate
 0353:02D2 idle  _PC_VectGet
 0353:02E5       _PC_VectSet
 0382:000E idle  _OSEventTaskRdy
 0382:00D8 idle  _OSEventTaskWait
 0382:0145 idle  _OSEventTO
 0382:0199 idle  _OSEventWaitListInit
 0382:01BD       _OSInit
 0382:032A idle  _OSIntEnter
 0382:0332       _OSIntExit
 0382:039D idle  _OSSched
 0382:03FD idle  _OSSchedLock
 0382:040C idle  _OSSchedUnlock
 0382:0435       _OSStart
 0382:0494       _OSStatInit
 0382:04CF idle  _OSTaskIdle
 0382:04EF idle  _OSTaskStat
 0382:05AA idle  _OSTCBInit
 0382:070E       _OSTimeTick
 0382:0799       _OSVersion
 0382:079D idle  _OSMboxAccept
 0382:07E2       _OSMboxCreate
 0382:0843       _OSMboxPend
 0382:096B       _OSMboxPost
 0382:09CB idle  _OSMboxQuery
 0382:0A42 idle  _OSQAccept
 0382:0AD4       _OSQCreate
 0382:0BE9 idle  _OSQFlush
 0382:0C36 idle  _OSQInit
 0382:0C6B       _OSQPend
 0382:0E04       _OSQPost
 0382:0EB3 idle  _OSQPostFront
 0382:0F5E idle  _OSQQuery
 0382:101A       _OSTaskCreateExt
 0382:1133 idle  _OSTaskStkChk
 0382:1218 idle  _OSTaskQuery
 0382:127B       _OSTimeDly
 0382:12C2       _OSTimeDlyHMSM
 0382:13B1 idle  _OSTimeDlyResume
 0382:142D idle  _OSTimeGet
 0382:144C idle  _OSTimeSet
 04C9:0306       e087_Entry
 04C9:03C6       e087_Shortcut
 04C9:0430       e087_Trap
 0526:0000 idle  DATASEG@
 0526:005B idle  __Int0Vector
 0526:005F idle  __Int4Vector
 0526:0063 idle  __Int5Vector
 0526:0067 idle  __Int6Vector
 0526:006B idle  __C0argc
 0526:006D idle  __C0argv
 0526:0071 idle  __C0environ
 0526:0075 idle  __envLng
 0526:0077 idle  __envseg
 0526:0079 idle  __envSize
 0526:007B       __psp
 0526:007D idle  __osversion
 0526:007D idle  __osmajor
 0526:007D       __version
 0526:007E idle  __osminor
 0526:007F       _errno
 0526:0081 idle  __StartTime
 0526:0085 idle  ___brklvl
 0526:0087       __heapbase
 0526:008B       __brklvl
 0526:008F       __heaptop
 0526:0296 idle  _OSMapTbl
 0526:029E idle  _OSUnMapTbl
 0526:03A0 idle  __8087
 0526:03B0       __protected
 0526:03B1       __LDT
 0526:03B4       __default87
 0526:04D0       __atexitcnt
 0526:04D2       __exitbuf
 0526:04D6 idle  __exitfopen
 0526:04DA idle  __exitopen
 0526:04DE       __streams
 0526:066E       __nfile
 0526:0670       __openfd
 0526:0698       __fpstklen
 0526:069A idle  __doserrno
 0526:069C idle  __dosErrorToSV
 0526:06F6       __stklen
 0526:0760       __wscroll
 0526:0762       __video
 0526:0771       _directvideo
 0526:07AE       __cFlag
 0526:07AF       __cChar
 0526:07B6       __RealCvtVector
 0526:07BA idle  __ScanTodVector
 0526:07D8 idle  _MsgQueueTbl
 0526:0828 idle  _MsgQueue
 0526:082C idle  _Task5Stk
 0526:0C2C idle  _Task4Stk
 0526:102C idle  _Task3Stk
 0526:142C idle  _Task2Stk
 0526:182C idle  _Task1Stk
 0526:1C2C idle  _TaskClkStk
 0526:202C idle  _TaskStartStk
 0526:242C idle  _TaskUserData
 0526:25A8       _OSTickDOSCtr
 0526:25AA idle  _PC_TickISR
 0526:341B idle  _OSTime
 0526:341F idle  _OSTCBPrioTbl
 0526:351F idle  _OSTCBList
 0526:3523       _OSTCBHighRdy
 0526:3527 idle  _OSTCBFreeList
 0526:352B       _OSTCBCur
 0526:352F       _OSTaskCtr
 0526:3530       _OSRunning
 0526:3531 idle  _OSRdyTbl
 0526:3539 idle  _OSRdyGrp
 0526:353A       _OSPrioHighRdy
 0526:353B       _OSPrioCur
 0526:353C idle  _OSLockNesting
 0526:353D       _OSIntNesting
 0526:353E idle  _OSStatRdy
 0526:353F idle  _OSIdleCtrRun
 0526:3543 idle  _OSIdleCtrMax
 0526:3547       _OSCPUUsage
 0526:3548 idle  _OSIdleCtr
 0526:354C idle  _OSEventTbl
 0526:368C idle  _OSEventFreeList
 0526:3690       _OSCtxSwCtr
 0526:3694       __atexittbl
 0526:3714       ___SignalPtr
 0898:0000       __emu

Program entry point at 0000:0000

